:100000008A011528FF280A2982073F3406345B3409
:100010004F3466346D347D3407347F346F34773435
:100020007C3439345E34793471348312860185012D
:10003000CF3083168500860180309F0051308312B7
:100040009F00AD0128308312AB0002208A110A12F2
:1000500083121F1583121F192A281E08A001A90048
:100060002008AA002908A1002A08A000A10DA00DBF
:10007000A10DA00DA10DA00DA10DA00DA10DA00D14
:10008000A10DA00DA10DA00DA10DA00D21080039FD
:10009000A10183161E078312A1000318A00A2108DC
:1000A000A9002008AA00AE0183122D082E020130FB
:1000B00003180301003C031986282A08A000290818
:1000C000A100A2010A30A3001030A400A501A601DE
:1000D0008312200DA60DA50D2308A6022208031CDD
:1000E000220FA50203187B282308A607220803185D
:1000F000220FA50703108312A10DA00DA40B6828E1
:100100002108A9002008AA00AE0A542883122A0850
:10011000A0002908A100A2010A30A3001030A40009
:10012000A501A6018312200DA60DA50D2308A60288
:100130002208031C220FA5020318A5282308A607DE
:1001400022080318220FA50703108312A10DA00D8A
:10015000A40B92282508A0002608AC002C088600D5
:10016000A0012D08043E0318A00AA000003C031DB6
:10017000BB280614EB2883122008013C031DC2286B
:100180008614EB2883122008023C031DC92806159B
:10019000EB2883122008033C031DD0288615EB288A
:1001A00083122008043C031DD7280616EB2883126F
:1001B0002008053C031DDE288616EB288312200844
:1001C000063C031DE5280617EB2883122008073C90
:1001D000031DEB288617033083122D02013003180C
:1001E0000301003C0319F628AD0AF8288312AD017B
:1001F00001308312A70003208A110A122228AB0CB7
:10020000AB0C3F30AB050330AB020000AB0B052954
:10021000000008008E308312A800000000000000DB
:10022000000000000000A80B0F290000A70B0A29FE
:0402300000000800C2
:00000001FF
